:020000040000FA
:100000000A128A11CC2A00008A0028080A3E031826
:100010008A0A820000340034003400340034003492
:1000200000342F34003400340034073400340734F3
:10003000003414347F3414347F34143424342A3498
:100040007F342A341234C434C8341034263446344D
:1000500036344934553422345034003405340334B2
:100060000034003400341C34223441340034003471
:10007000413422341C340034143408343E340834FF
:100080001434083408343E3408340834003400345E
:1000900050343034003410341034103410341034F0
:1000A00000346034603400340034203410340834B8
:1000B000043402343E345134493445343E3400343F
:1000C00042347F3440340034423461345134493452
:1000D00046342134413445344B34313418341434EB
:1000E00012347F34103427344534453445343934A0
:1000F0003C344A344934493430340134713409349D
:1001000005340334363449344934493436340634FA
:100110004934493429341E340034363436340034FA
:100120000034003456343634003400340834143487
:100130002234413400341434143414341434143458
:10014000003441342234143408340234013451343C
:100150000934063432344934593451343E347E340F
:100160001134113411347E347F34493449344934E4
:1001700036343E3441344134413422347F344134C6
:10018000413422341C347F344934493449344134B5
:100190007F3409340934093401343E34413449345C
:1001A00049347A347F340834083408347F340034D6
:1001B00041347F34413400342034403441343F34BE
:1001C00001347F3408341434223441347F344034D1
:1001D0004034403440347F3402340C3402347F34B1
:1001E0007F340434083410347F343E344134413495
:1001F00041343E347F3409340934093406343E3402
:100200004134513421345E347F3409341934293473
:1002100046344634493449344934313401340134A4
:100220007F34013401343F344034403440343F346F
:100230001F342034403420341F343F3440343834A9
:1002400040343F3463341434083414346334073492
:100250000834703408340734613451344934453437
:10026000433400347F3441344134003455342A342B
:1002700055342A3455340034413441347F34003409
:100280000434023401340234043440344034403401
:100290004034403400340134023404340034203417
:1002A00054345434543478347F34483444344434EB
:1002B00038343834443444344434203438344434C6
:1002C000443448347F343834543454345434183437
:1002D00008347E340934013402340C34523452343C
:1002E00052343E347F3408340434043478340034D7
:1002F00044347D34403400342034403444343D347C
:1003000000347F3410342834443400340034413411
:100310007F34403400347C3404341834043478346A
:100320007C34083404340434783438344434443469
:10033000443438347C3414341434143408340834D9
:100340001434143418347C347C34083404340434C5
:1003500008344834543454345434203404343F344E
:100360004434403420343C344034403420347C34F1
:100370001C342034403420341C343C344034303479
:1003800040343C34443428341034283444340C345D
:100390005034503450343C344434643454344C3449
:1003A0004434820720342A342034453452344134D2
:1003B00053344534203445344534503452344F346A
:1003C0004D3420344D3445344D344F345234593447
:1003D00020342A34203482072A342034353420341F
:1003E0006B34573420342A3482072A3432342E3482
:0A03F000353420346B3457342A34BE
:10040000820749344E3420342034203420342034C0
:10041000203420342034203420342034203420343C
:10042000203420344F345534543420342034203494
:10043000203420348207503452344F3447345234FD
:1004400041344D342034623461347334653464345F
:1004500020346F346E3420344A3441344C344C34BC
:1004600049344234203482072A342A342A342A3444
:10047000203453344D3441345234543420344D34C8
:10048000453454344534523420342A3431343034F1
:100490002A342A342A342A3482072A342A342A3441
:1004A0002A342A342A342034483461346E347A347D
:1004B00065346D3461346E3420342A342A342A345D
:1004C0002A342A34383465342A34820720344F34AD
:1004D0005534543482074F346D3461347834820794
:1004E00049346D34613478348207203449344E34D1
:1004F0002E34820720344E3472342E341030A8004B
:100500000310A40DA50D0310A00DA10D031C8E2A30
:100510002308A5072208A4070318A50AA80B802A08
:1005200008001030A800A201A3010310A60DA70D1A
:100530000310A00DA10DA20DA30D23082502031D7C
:10054000A32A220824020319A72A0318AE2A250881
:10055000A3022408A202031CA3032614A80B952AB5
:1005600008008000840AA80BB12A0800AB1BC72A28
:100570002B1BC22A2A0884008313AB08031D831790
:10058000000808002A08A9002B083F39C82A0800DB
:100590008A0003132A08820083134F3084002A3014
:1005A000A8000030B1228313A030840050308312A1
:1005B0000313A80000308A110A12B12283171030E9
:1005C0008400443083120313A80000308A110A12F9
:1005D000B1228A110A12831203139F010730831676
:1005E0009F0007309C002B2B813083169900181533
:1005F0000800980183129801F422831603138C12C9
:100600000C128717071798168312981718160800E8
:10061000831203179D0003130C1A0F2B0B2B0317C8
:100620001D0803139900080083128C1E1D2B1A0845
:100630008316B40083128C12202B83163810262BBD
:10064000981C242B18121816831638143818292BC6
:10065000142B34080800F9228316031307118312A0
:10066000AC010130AD008A110A12602B8316B40070
:100670008312AC010130AD002C03831692003403C9
:10068000031D472BFC30831292051215080004301D
:100690003402031D522BFC308312120501389200E4
:1006A0001215080010303402031D5D2BFC3083123C
:1006B0001205023892001215080083121211080068
:1006C000CF01D001072CF0308312031350050C38F2
:1006D000D0004F089500500897000800033017021B
:1006E000031D742BFF30160203197C2B031C7C2B7B
:1006F000FF309600033097000310170C0313A1007E
:100700000317160C0313A0000310A10CA00C200863
:10071000CF000330031716050313A000200EA1001D
:100720003030A105CF3050052104D000632B831653
:100730000313CF004F08031DA02BD701D801F22BC4
:1007400064304F020319A62B031CB22B83122D0811
:100750008316D80083122C038316D700570A031977
:10076000D803F22B4F08DF00E001031083122D0C99
:100770008316E20083122C0C8316E1000310E20CB6
:10078000E10C5F088312A000831660088312A100A9
:10079000831661088312A200831662088312A300E5
:1007A0007E228312031324088316E3008312250894
:1007B0008316E40019308312A400A5018316630890
:1007C0008312A000831664088312A1008A110A1202
:1007D00091228312031326088316D7008312270859
:1007E0008316D8000310570DDF00580DE0000310EA
:1007F000DF0DE00D5F0883120317960083160313C5
:1008000060088312031797008A110A126E2B0130B9
:1008100036238A110A12632332308A110A1297236F
:100820008316031305160514851405158A110A127B
:10083000682D25088D0026088F0083168C170C1450
:100840000000000083120C08AB000E08AC0008008A
:100850001D08A5001E08A6001924831203172B08E3
:10086000A1002C08A20021080313A00003172208EE
:100870000313A1000800831203171C108B1B1C1408
:10088000FC30831603133F05C9004008CA00EE017F
:1008900003106E0D831203179600831603134A0884
:1008A000831203179800831603136E0849078312F7
:1008B000031797000318980A17089D0018089E0050
:1008C0002824CF30831203171607840083130313E1
:1008D00020088000840A210880008316EE0A043074
:1008E0006E028A110A12031D482C03303F05831241
:1008F0000317960097010310160D9800170D990025
:10090000CF30180784008313831603134508800033
:10091000840A460880004908831203178D00831655
:1009200003134A08831203178F0083160313EE0183
:1009300003106E0D831203179600CF301607840044
:100940008313000883160313C500840A0008C60039
:100950004508831203178C0083160313460883127D
:1009600003178E0083168C170C158B1355308D00D2
:10097000AA308D008C14000000000C1183128D0A27
:1009800083160313EE0A04306E02031D982C8312A3
:1009900003171C18CD2C8B1308008B1708001D089B
:1009A000A1001E08A200A501A601E92C83120313D1
:1009B0000630A000A530A1000A128A11A10BDC2C80
:1009C0000A128A11A00BDA2C00000317A50A0319DA
:1009D000A60A250821020313A000031726082202F5
:1009E00003132004031DD62C08001F08A3002008B1
:1009F000A400A701A801152D831203135E30A000E7
:100A0000FD30A1000330A2000A128A11A20B042DAE
:100A10000A128A11A10B022D0A128A11A00B002DB5
:100A200000000317A70A0319A80A270823020313C3
:100A3000A00003172808240203132004031DFC2C24
:100A400008002308AD002408AE002D08B3002E08CE
:100A5000B400B101462D031728080313AB00031798
:100A6000310827070313AA000318AB0AB622831222
:100A70000313A00003171F080313AA00031720087D
:100A80008A110A12C82283120317B10A31083302ED
:100A90000313A00003173408031320048A110A1259
:100AA000031D2B2D0800B4003403031D5C2D013001
:100AB0008312D1000530D20083163408340A0800AE
:100AC0005103031D672D4D08A8004E08042800346B
:100AD0000130532583120313D3010130D4008A154A
:100AE0000A1238290313C900FC127C088600000092
:100AF00000000000000000004A18822D7C147C08D1
:100B00008600852DFC147C0886007C127C088600FB
:100B1000000000000000000000004908FA007A0808
:100B2000880083168801FC167C088312860000006A
:100B300000000000000000000000000000000000B5
:100B40000000FC127C08860000000000000000008D
:100B500000007C107C088600FC107C0886000800E1
:100B6000FC127C088600000000000000000000006D
:100B70004C18BE2D7C147C088600C12DFC147C080A
:100B800086007C167C088600000000000000000043
:100B90000000FC167C088600000000000000000039
:100BA000000000000000000000000000FC127C08B3
:100BB000860000000000000000000000FF308316E7
:100BC000880083120808CB007C107C088600FC108B
:100BD0007C0886004B080800831203134A103F303C
:100BE0007225831203134A143F308A110A12722DA0
:100BF000C9005110403049020319002E031C032E76
:100C00004030C90251147C117C0886003F304905F0
:100C1000D20040305204D3005118112E03134A1051
:100C2000132E03134A14031753087225031083125B
:100C300003174A0CCF000310CF0C0310CF0C073062
:100C40004F05D200B8305204D3008A110A1251184D
:100C50002C2E03134A102E2E03134A140317530885
:100C600072257C157C088312860003178A110A12EC
:100C700051183D2E03134C103F2E03134C14B02576
:100C800083120317CB008A110A1251184A2E03133C
:100C90004C104C2E03134C14B02583120317CB00B9
:100CA000031354038A110A12031D672E073003171A
:100CB0004A05CC00FF000130CD007F08622E0310F2
:100CC000CD0DFF03031D5F2E4D08CB04782E07309A
:100CD00003174A05CC00FF000130CD007F08732EBA
:100CE0000310CD0DFF03031D702E4D09CE00CB0563
:100CF0007C117C0886003F304905D2004030520408
:100D0000D3005118862E03134A10882E03134A1459
:100D10000317530872250310831203174A0CD000DF
:100D20000310D00C0310D00C07305005D200B8309F
:100D30005204D3008A110A125118A12E03134A102B
:100D4000A32E03134A140317530872257C157C083D
:100D50008312860003178A110A125118B22E031348
:100D60004A10B42E03134A1403174B08722DBA000D
:100D7000411040303A020319BF2E031CC22E4030EE
:100D8000BA0241147C117C0886003F303A05C2004B
:100D900040304204C3004A1041184A1443087225E7
:100DA0000310831203133B0CC0000310C00C03108C
:100DB000C00C07304005C200B8304204C3004A10DE
:100DC00041184A1443088A110A1272257C157C08BE
:100DD00083128600073003133B05BD003D088A11CE
:100DE0000A12031DF82E4A1041184A143C08722DAD
:100DF0004C1041184C14B02583120313C2004C1040
:100E000041184C148A110A12B02583120313C20030
:100E100007303B05BD003D09BE000930BE073E0856
:100E2000FF00FF30BF00FF088A110A1203191C2FB0
:100E30000310BF0CFF0B182F3F08C20507303B05FE
:100E4000BD00FF003C08BE007F08292F0310BE0D27
:100E5000FF03031D262F3E08C2047C117C08860078
:100E60003F303A05C60040304604C7004A104118DA
:100E70004A14470872250310831203133B0CC30066
:100E80000310C30C0310C30C07304305C600B83071
:100E90004604C7004A1041184A1447088A110A122A
:100EA00072257C157C088312860003134A104118B2
:100EB0004A1442088A110A1272257C117C08831296
:100EC00086003F3003133A05C60040304604C70091
:100ED0004A1041184A1447088A110A127225031051
:100EE000831203133B0CBD000310BD0C0310BD0C9B
:100EF0003D0AC40007304405C600B8304604C700A8
:100F00004A1041184A1447088A110A1272257C15A2
:100F10007C088312860003134C1041184C148A116C
:100F20000A12B02583120313C2004C1041184C144E
:100F30008A110A12B02583120313C20007303B0541
:100F4000BD00FF00FF30BE007F088A110A12AB2FE0
:100F50000310BE0DFF03031DA82F3E08C205073076
:100F60003B05BD003D09BE000930BE073E08FF003D
:100F70003C08BF00FF080319C12F0310BF0CFF0B73
:100F8000BD2F3F08C2047C117C0886003F303A0523
:100F9000C60040304604C7004A1041184A144708AA
:100FA00072250310831203133B0CBD000310BD0C0C
:100FB0000310BD0C3D0AC50007304505C600B8301A
:100FC0004604C7004A1041184A1447088A110A12F9
:100FD00072257C157C088312860003134A10411881
:100FE0004A1442088A110A12722D0317A500A7019C
:100FF0007C117C08860007302705AD00B8302D0431
:10100000AE0003134A1003172E087225073083120F
:1010100003172705AD00B8302D04AE0003134A14A2
:1010200003172E088A110A12722583120317AD01C5
:101030003F302D05AF0040302F04B00003134A109D
:10104000031730088A110A12722583120317AD01A3
:101050003F302D05AF0040302F04B00003134A1479
:10106000031730088A110A1272257C157C08831236
:1010700086000317AB0103134A10031725088A11D2
:101080000A127225831203134A14031725088A11C2
:101090000A12722583120317AB0A80302B028A15BD
:1010A0000A12031D3B28A70A083027028A11031DD4
:1010B000F82F08007B107B088312031387000000C1
:1010C0000000000000000000000000000000000020
:1010D00000007B147B0887005308031D752800302F
:1010E0008A11F5278A150A127828FF308A11F52708
:1010F0007C117C088312860003179F0107301F05AF
:10110000A100B8302104A20003134A1003172208DB
:101110008A110A127225831203179F0107301F05D7
:10112000A100B8302104A20003134A1403172208B7
:101130008A110A127225831203179F013F301F057F
:10114000A10040302104A20003134A100317220813
:101150008A110A127225831203179F013F301F055F
:10116000A10040302104A20003134A1403172208EF
:101170008A110A1272258A110A12EC2DFA017A08D4
:101180008800831688017C157C08831286007C12F7
:101190007C088600FC167C0886007C107C08860093
:1011A000FC107C0886007B147B08870083160612DF
:1011B000061186120610861007105A28AF0020303C
:1011C000310239100319E628031C39147A30310230
:1011D000B9100319ED280318B9143911391CB918BD
:1011E0003915391DF5282030B10020303102B50005
:1011F000B6015208A000A1013508A2003608A300DC
:101200008A117E22831203132408B2002508B3003A
:101210005208B700B8018A150A12312980302F020E
:1012200003191429031C152908003208CD003308BE
:10123000CE008A11602583120313B40054088A1566
:101240000A120319B4093008BB003408BC002F0887
:101250008A11B72683120313B20A0319B30AAF0A1D
:10126000B80A380837028A150A12031D0E29080029
:10127000D501D601712A831203132008AE00560847
:10128000B0002E08B10055088A150A12DE2083121C
:1012900003135208D5070800831203179F00230881
:1012A000A700A8011F08A900AA012A082802B20065
:1012B00029082702B100031CB2032508A700A801D2
:1012C0002108A900AA012A082802B6002908270235
:1012D000B500031CB6030310310DB700320DB80082
:1012E0000310350DB900360DBA001F08BB00BC0154
:1012F0002108BD00BE010130BF00C0010130C100A6
:10130000C2013208803A0313A00080302002031D7E
:101310008C2900300317310203199E2903189E29D6
:10132000FF300317BF00C000B109B209B10A0319A9
:10133000B20AB709B809B70A0319B80A0317360879
:10134000803A0313A00080302002031DAA29003038
:10135000031735020319BC290318BC29FF300317F2
:10136000C100C200B509B609B50A0319B60AB90920
:10137000BA09B90A0319BA0A03172108CA001F08D3
:101380008A11F8258312031731083204471503190F
:10139000471135083604C7150319C7114712471DF1
:1013A000C71947168A150A12471E702A3208803A52
:1013B0000313A00003173608803A03132002031D0D
:1013C000E4290317350831020319E829031C2C2AE4
:1013D0000317C301C401831203173B08230203133D
:1013E000A00003173C08031320040319702A0317F5
:1013F0004008BC073F08BB070318BC0A3A08C407EB
:101400003908C3070318C40A3208803A0313A0003E
:1014100003174408803A03132002031D122A0317FE
:10142000430831020319232A0318232A0317420809
:10143000BE074108BD070318BE0A3808C4023708B2
:10144000C302031CC40303173D08CA003B088A11EA
:10145000F8258A150A12EB290317C501C601831264
:1014600003173D0825020313A00003173E080313CA
:1014700020040319702A03174208BE074108BD075C
:101480000318BE0A3808C6073708C5070318C60A76
:101490003608803A0313A00003174608803A031366
:1014A0002002031D562A0317450835020319672A2F
:1014B0000318672A03174008BC073F08BB07031837
:1014C000BC0A3A08C6023908C502031CC603031742
:1014D0003D08CA003B088A11F8258A150A122F2AEE
:1014E0000800BE20303083120313D7003130D800FB
:1014F0003230D9003330DA002E30DB003430DC00FB
:101500003530DD003030DE003630DF003230E000D4
:101510003130E1002E30E2003830E3003630E400B4
:10152000EB01EC01F101F201F301F401F501F60127
:10153000F701D3010530F80005308316A40005300B
:10154000A5008A110A16C62B5A20013083120313F4
:10155000D400F501F601750883120313A000760884
:10156000A1000A30A200A3018A110A127E2283126E
:10157000031324088316E600831225088316E70068
:10158000E90004306607E8000318E90A831224081A
:101590008316EA00831225088316EB00ED00043061
:1015A0006A07EC000318ED0A183083120317A10034
:1015B000831603136C0883120317A3001A30A500C7
:1015C0008316031368088A150A124C21F50A0319B9
:1015D000F60A0D30750276048A150A12031DAB2A2D
:1015E000323083120317A1007E30A300A5017E30A4
:1015F0004C21F501F601750883120313A00076084B
:10160000A1000530A200A3018A110A127E228312D2
:10161000031324088316E600831225088316E700C7
:10162000831224088316E800831225088316E90034
:10163000660883120317A1007E30A30083160313EC
:10164000680883120317A5007C308A150A124C2102
:10165000F50A0319F60A0B30750276048A150A1288
:10166000031DFB2A0130F500F601831203179C01CC
:1016700037309D001C080313D50003171D08031302
:10168000D6003B3003179F000930A0001930A3009B
:10169000A4010130A70002304038A8008A1121259A
:1016A0000130831203179F00A0018A110A12F52C42
:1016B0008A11142383120313E5007F30E505080027
:1016C00083160313B401B501831269086A048316F3
:1016D0004B14031D4B108312670868048316CB1448
:1016E0000319CB104B154B18CB1C4B1183126908F7
:1016F0006A048316CB150319CB118312670868049B
:1017000083164B16031D4B12CB16CB194B1ECB1257
:101710004B134B1DCB1A4B174B1FC62B0A30831292
:10172000A400A5016908A0006A08A1008A119122FD
:101730008312031326088316B90083122708831621
:10174000BA00BC0032303907BB000318BC0A0A30AB
:101750008312A400A5016708A0006808A1008A11EF
:101760000A1291228312031326088316BD008312E6
:1017700027088316BE003C02B5003D083B02B400BA
:10178000031CB50334088A110A12972B08009B002A
:101790000530CA001B088A11F82583120317A1011E
:1017A0001B08A3000330A5001B088A150A124C2948
:1017B000013083120313D400F501F6018316E6010C
:1017C00076088312031791007508770790000318B5
:1017D000910AF0300313A400A501031710080313A6
:1017E000A000031711080313A1008A11912283128C
:1017F000031322088316A000831223088316A10076
:101800001B30A1075830A0070318A10A2008831233
:1018100003179D00831603132108831203179E00EC
:101820008A110A1228248312031320088316A200A7
:10183000831221088316A30078088312A400A5014F
:10184000831622088312A000831623088312A100A6
:101850008A110A1291228312031326088316A2000A
:10186000831227088316A300003023028A150A1268
:10187000031D3C2C323022020319422C031C422C43
:10188000A201A30100302302031D482C1C302202B8
:1018900003195B2C031C5B2C1930A200A3017509F2
:1018A000831203179000760991007D30900703188A
:1018B000910A1008C723750983120317900076094F
:1018C00091007D3090070318910A831603132308B3
:1018D0008312031793001930831603132207831210
:1018E000031792000318930A75099400760995006E
:1018F0007D3094070318950A1208A1001408A3006C
:101900001930A50010088A150A124C2101308316DF
:101910000313A107E030A0070318A10A20088312CF
:1019200003179D00831603132108831203179E00DB
:101930008A110A1228248312031320088316A20096
:10194000831221088316A30078088312A400A5013E
:10195000831622088312A000831623088312A10095
:101960008A110A1291228312031326088316A200F9
:10197000831227088316A300003023028A150A1257
:10198000031DC42C193022020319D62C031CD62C9B
:10199000A201A30175098312031790007609910033
:1019A0007D3090070318910A1008C7237509831228
:1019B00003179000760991007D3090070318910A73
:1019C000831603132209831203179200831603134D
:1019D00023098312031793001A3092070318930AFE
:1019E00075099400760995007D3094070318950ACF
:1019F0001208A1001408A3001930A50010088A15C8
:101A00000A124C21F50A0319F60A83160313E60A93
:101A1000783066028A150A12031DE02B08005A0866
:101A20008316B40083125B088316B50083125C082A
:101A30008316B60083125D088316B7003408C10010
:101A40003508C2003608C3003708C4000F30DF0075
:101A50003730E5005F088312D500831665088312CE
:101A6000D6003B3003179F000930A0000430A300CC
:101A7000A401C130A700A8018A11212583120313F4
:101A800061088316B400831262088316B5008312BE
:101A900063088316B600831264088316B7003408FF
:101AA000CB003508CC003608CD003708CE006930B1
:101AB000DF003730E5005F088312D5008316650824
:101AC0008312D6003B3003179F000930A00004307A
:101AD000A300A401CB30A700A8018A110A12212576
:101AE000283083160313DF003730E5005F088312C8
:101AF000D500831665088312D6008A150A12851848
:101B0000952D0530F8003B3003179F000930A000E9
:101B10000830A300A401F530A70001304038A80028
:101B20008A1121258A150A12A62D0A30F8003B30A9
:101B300003179F000930A0000830A300A401EC3077
:101B4000A70001304038A8008A11212578088316A3
:101B5000031324028A150A120319B42D7808A4006D
:101B6000A4228A150A12D823831203138A150A1293
:101B70000519BE2D23308316A500080005308316F5
:101B8000A5000800573083120317A5001B30A600DC
:101B90008A111924831203172B08F70083160313E5
:101BA0003914031D3910EF307702B9108A150A1263
:101BB0000319DC2D0318B9143911391CB91839155A
:101BC000391DE52DEF30F700E62DF7035730BF0044
:101BD0001B30C0007708C500C6018A113B240310E2
:101BE000F20CF10C003072028A150A12031DFA2D54
:101BF000FF3071020319012E031C012EFF30F1008A
:101C0000F2010310F40CF30C00307402031D0A2ED1
:101C1000FF3073020319112E031C112EFF30F30045
:101C2000F401831203136B08A4006C08A5006D086F
:101C3000A0006E08A1008A119122831203132608C6
:101C40008316B400831227088316B5000310350CE1
:101C50008312EE008316340C8312ED0000306E0206
:101C60008A150A12031D362EFF306D0203193D2E10
:101C7000031C3D2EFF30ED00EE016B08A4006C0844
:101C8000A5006F08A0007008A1008A11912283129C
:101C9000031326088316B400831227088316B500A1
:101CA0000310350C8312F0008316340C8312EF00FE
:101CB000003070028A150A12031D602EFF306F0279
:101CC0000319672E031C672EFF30EF00F0011B3055
:101CD0008316A10058307707A0000318A10A200836
:101CE000BF002108C00083126D088316C50083124F
:101CF0006E088316C6008A113B24F0308316031346
:101D0000A0070318A10A2008BF002108C00071081D
:101D1000C5007208C6008A110A123B24F0308316EF
:101D20000313A0070318A10A2008BF002108C00060
:101D300083126F088316C500831270088316C600CD
:101D40008A110A123B24F03083160313A0070318EC
:101D5000A10A2008BF002108C0007308C50074084C
:101D6000C6008A110A123B248A150A12A4228A1577
:101D70000A12D82383120313EB01EC01ED01EE01EB
:101D8000EF01F001E701E801E901EA01F101F201E7
:101D9000F301F401080057300317A5001B30A6001B
:101DA0008A111924831203172B08F70083160313D3
:101DB000CB01CC01D70102308A004B088A110A12EC
:101DC0004C228A110A12082383160313CB0A031923
:101DD000CC0AD70A103057028A150A12031DDB2ECF
:101DE0000D308A1108230A308A110A12082383163B
:101DF0000313CB01CC01EE0102308A004B088A119B
:101E00000A1279228A110A12082383160313CB0AB5
:101E10000319CC0AEE0A04306E028A150A12031D59
:101E2000FC2E09308A11082383160313CB01CC0141
:101E300083120317960102308A00831603134B089E
:101E40008A110A1274228A110A12082383160313B4
:101E5000CB0A0319CC0A83120317960A0430160220
:101E60008A150A12031D1B2F09308A1108238316B5
:101E70000313CB01CC01EF0102308A004B088A1119
:101E80000A126F228A110A12082383160313CB0A3F
:101E90000319CC0AEF0A04306F028A150A12031DD7
:101EA0003C2F09308A11082383160313CB01CC0180
:101EB000831203179A0102308A00831603134B081A
:101EC0008A110A1265228A110A1208238316031343
:101ED000CB0A0319CC0A831203179A0A04301A0298
:101EE0008A150A12031D5B2F09308A1108238316F5
:101EF0000313CB01CC01831203179B0102308A002C
:101F0000831603134B088A110A126A228A110A12D5
:101F1000082383160313CB0A0319CC0A8312031771
:101F20009B0A04301B028A150A12031D7E2F0930FA
:101F30008A1108230D308A110A1208230A308A11E7
:101F40000A120823F03083160313CB00CC0183124E
:101F500003179C01831603134C08DA004B0877071C
:101F6000D9000318DA0AF0308312A400A501831601
:101F700059088312A00083165A088312A1008A11FF
:101F80000A1291228312031322088316A0008312DF
:101F900023088316A1001B30A1075830A00703189F
:101FA000A10A2008831203179D008316031321083A
:101FB000831203179E008A110A1228248312031326
:101FC00020088316B400831221088316B50003107D
:101FD000B40DB50D033035028A150A12031DF22F18
:101FE000E73034020319FA2F031CFA2FE730B4004C
:101FF0000330B500F030A0070318A10A20088312AF
:1020000003179D00831603132108831203179E00F4
:102010008A1128248312031320088316B90083121F
:1020200021088316BA000310B90DBA0D03303A0225
:102030008A110A16031D1E28E730390203192628C3
:10204000031C2628E730B9000330BA00F030A0079F
:102050000318A10A2008831203179D008316031397
:102060002108831203179E000A12282483120313E7
:1020700020088316C100831221088316C2000310B2
:10208000C10DC20D033042028A110A16031D4A28EF
:10209000E730410203195228031C5228E730C100DF
:1020A0000330C200F030A0070318A10A20088312F1
:1020B00003179D00831603132108831203179E0044
:1020C0000A1228248312031320088316C7008312E0
:1020D00021088316C8000310C70DC80D033048023D
:1020E0008A110A16031D7628E730470203197E2855
:1020F000031C7E28E730C7000330C800E830831295
:10210000A4000330A50083164B088312A000831699
:102110004C088312A1000A12912283120313220891
:102120008316D900831223088316DA0064308312E1
:10213000A400A501831659088312A00083165A082B
:102140008312A1008A110A12912283120313260816
:102150008316DB00831227088316DC00DE00303094
:102160005B07DD000318DE0A5D088A110A120823E6
:10217000643083120313A400A50183164B08831255
:10218000A00083164C088312A1008A110A12912222
:102190008312031322088316D9008312230883169F
:1021A000DA000A308312A400A501831659088312AD
:1021B000A00083165A088312A1008A110A129122E4
:1021C0008312031326088316DB0083122708831665
:1021D000DC00DE0030305B07DD000318DE0A5D083E
:1021E0008A110A1208230A3083120313A400A501DE
:1021F00083164B088312A00083164C088312A1009B
:102200008A110A1291228312031322088316D9001D
:10221000831223088316DA00DC0030305907DB0014
:102220000318DC0A5B088A110A12082309308A1194
:102230000A1208232D308A110A120823E83083126B
:102240000313A4000330A500831634088312A000F2
:10225000831635088312A1008A110A129122831273
:10226000031322088316D900831223088316DA0089
:1022700064308312A400A501831659088312A000BC
:1022800083165A088312A1008A110A12912283121E
:10229000031326088316DB00831227088316DC004D
:1022A000DE0030305B07DD000318DE0A5D088A11AE
:1022B0000A1208232C308A110A1208236430831270
:1022C0000313A400A501831634088312A00083160B
:1022D00035088312A1008A110A1291228312031376
:1022E00022088316D900831223088316DA000A30E5
:1022F0008312A400A501831659088312A000831637
:102300005A088312A1008A110A1291228312031320
:1023100026088316DB00831227088316DC00DE0004
:1023200030305B07DD000318DE0A5D088A110A12EF
:1023300008230A3083120313A400A501831634086E
:102340008312A000831635088312A1008A110A1295
:1023500091228312031322088316D90083122308C3
:102360008316DA00DC0030305907DB000318DC0A82
:102370005B088A110A12082309308A110A120823FD
:102380002D308A110A120823E83083120313A400A7
:102390000330A500831639088312A00083163A087B
:1023A0008312A1008A110A129122831203132208B8
:1023B0008316D900831223088316DA00643083124F
:1023C000A400A501831659088312A00083165A0899
:1023D0008312A1008A110A12912283120313260884
:1023E0008316DB00831227088316DC00DE00303002
:1023F0005B07DD000318DE0A5D088A110A12082354
:102400002C308A110A120823643083120313A400AB
:10241000A501831639088312A00083163A08831297
:10242000A1008A110A129122831203132208831633
:10243000D900831223088316DA000A308312A4001D
:10244000A501831659088312A00083165A08831227
:10245000A1008A110A1291228312031326088316FF
:10246000DB00831227088316DC00DE0030305B07B8
:10247000DD000318DE0A5D088A110A1208230A30FB
:1024800083120313A400A501831639088312A00048
:1024900083163A088312A1008A110A12912283122C
:1024A000031322088316D900831223088316DA0047
:1024B000DC0030305907DB000318DC0A5B088A11A6
:1024C0000A12082309308A110A120823E8308312FD
:1024D0000313A4000330A500831641088312A00053
:1024E000831642088312A1008A110A1291228312D4
:1024F000031322088316D900831223088316DA00F7
:1025000064308312A400A501831659088312A00029
:1025100083165A088312A1008A110A12912283128B
:10252000031326088316DB00831227088316DC00BA
:10253000DE0030305B07DD000318DE0A5D088A111B
:102540000A1208232C308A110A12082364308312DD
:102550000313A400A501831641088312A00083166B
:1025600042088312A1008A110A12912283120313D6
:1025700022088316D900831223088316DA000A3052
:102580008312A400A501831659088312A0008316A4
:102590005A088312A1008A110A129122831203138E
:1025A00026088316DB00831227088316DC00DE0072
:1025B00030305B07DD000318DE0A5D088A110A125D
:1025C00008230A3083120313A400A50183164108CF
:1025D0008312A000831642088312A1008A110A12F6
:1025E00091228312031322088316D9008312230831
:1025F0008316DA00DC0030305907DB000318DC0AF0
:102600005B088A110A12082309308A110A1208236A
:10261000E83083120313A4000330A5008316470893
:102620008312A000831648088312A1008A110A129F
:1026300091228312031322088316D90083122308E0
:102640008316DA0064308312A400A50183165908AA
:102650008312A00083165A088312A1008A110A125D
:1026600091228312031326088316DB0083122708A6
:102670008316DC00DE0030305B07DD000318DE0A65
:102680005D088A110A1208232C308A110A120823C5
:10269000643083120313A400A50183164708831234
:1026A000A000831648088312A1008A110A12912201
:1026B0008312031322088316D9008312230883167A
:1026C000DA000A308312A400A50183165908831288
:1026D000A00083165A088312A1008A110A129122BF
:1026E0008312031326088316DB0083122708831640
:1026F000DC00DE0030305B07DD000318DE0A5D0819
:102700008A110A1208230A3083120313A400A501B8
:10271000831647088312A000831648088312A1007D
:102720008A110A1291228312031322088316D900F8
:10273000831223088316DA00DC0030305907DB00EF
:102740000318DC0A5B088A110A1208230D308A116B
:102750000A1208230A308A110A1208238316031367
:10276000CB034B0A0319CC030A30831203179D00D5
:102770009E018A110A12CF24831203179C0AF0309B
:102780001C028A150A12031DAA2F08000A308312A0
:1027900003179F00A0010A12F524013083120313CE
:1027A000D4008A150A125A20023083160313AF0090
:1027B0000A30B1002F088312D50083163108831226
:1027C000D6003B3003179F000930A0001830A3004B
:1027D000A4014D30A70002304038A8008A110A1227
:1027E00021250A30831203179D009E018A110A12C7
:1027F000CF24023083160313AF001930B1002F0825
:102800008312D500831631088312D6003B3003179C
:102810009F000930A0001830A300A4013430A700A5
:1028200002304038A8008A110A1221250A3083128A
:1028300003179D009E018A110A12CF2402308316CD
:102840000313AF003230B1002F088312D500831676
:1028500031088312D6003B3003179F000930A000D7
:102860001830A300A4011B30A70002304038A80094
:102870008A110A1221251430831203179F00A00128
:102880008A110A12F52483160313A601F501F60135
:102890000310750D83160313A700760DA80003100F
:1028A000750DA900760DAA002909AB002A09AC0014
:1028B0008130AB070318AC0A2C08AE002B03AD0027
:1028C0002D0A0319AE0383120317A1018316031304
:1028D0002D0883120317A3003F30A50083160313AE
:1028E00027088A150A124C210A30831203179D000B
:1028F0009E018A110A12CF24F50A0319F60A3F3005
:10290000750276048A110A16031D482CF501F6019A
:10291000750983160313A7007609A8004130A7079D
:102920000318A80A750883120317A100A3018316D0
:102930000313270883120317A5007F308A150A1294
:102940004C210A30831203179D009E018A110A123E
:10295000CF24F50A0319F60A3F30750276048A116E
:102960000A16031D882C83120313D4018316A60AAA
:1029700002302602031D462C0A30831203179F00E3
:10298000A0010A12F5248A150A125A208312031391
:102990008A110A160518222D0130D4000230831640
:1029A000B2001930B30032088312D5008316330801
:1029B0008312D6003B3003179F000930A000193066
:1029C000A300A401D230A70001304038A8000A12A9
:1029D00021250A30831203179D009E018A110A12D5
:1029E000CF245730F5001B30F60083160313AF01D8
:1029F000B00175088316BF007608C000FF30C5001F
:102A0000C6018A110A123B24F50A0319F60A831635
:102A10000313AF0A0319B00ACA302F028312A000B1
:102A2000033083163002831220048A110A16031D14
:102A3000F92C0A3003179D009E010A12CF248A1533
:102A40000A125A208A150A12A4228A150A12D823B9
:102A50003A308312031365028A110A160319362DC0
:102A60008A150A1258238A110A16282D8A150A1265
:102A7000582331308312031365028A110A16031D8D
:102A8000452E8A150A1258232E308312031365022D
:102A90008A110A16031D452E8A150A12582337304B
:102AA0008312031365028A110A16031D452E8A1527
:102AB0000A1258232E308312031365028A110A1654
:102AC000031D452E8A150A12582330308312031332
:102AD00065028A110A16031D452E8A150A1258230B
:102AE00028308312031365028A110A16031D452E2E
:102AF000E6018316AF018A150A1258235730831254
:102B0000031366078400831365088000E60A8316B2
:102B1000AF0A07302F028A110A16031D7B2D2830B9
:102B200083120313650203199B2D8A150A12582379
:102B30008A110A168F2DE6018316B1018A150A1231
:102B400058235E30831203136607840083136508DD
:102B50008000E60A8316B10A073031028A110A168C
:102B6000031D9E2D303083125A028316A700831254
:102B7000A000A1016430A200A3010A127E228312E8
:102B8000031324088316A800303083125C028316D6
:102B9000A9008312A000A1010A30A200A3018A119A
:102BA0000A127E228312031324088316AA00280720
:102BB000AB00303083125D028316AC002B0783120A
:102BC000E700E801303061028316A7008312A000FD
:102BD000A1016430A200A3018A110A127E2283128D
:102BE000031324088316A80030308312630283166F
:102BF000A9008312A000A1010A30A200A3018A113A
:102C00000A127E228312031324088316AA002807BF
:102C1000AB003030831264028316AC002B078312A2
:102C2000E900EA016808EE076708ED070318EE0AF5
:102C30006A08F0076908EF070318F00AEB0A03199E
:102C4000EC0A720868028A110A16031D292E7108FF
:102C500067020319312E031C312E6708F100680842
:102C6000F20074086A02031D372E73086902031903
:102C70003F2E031C3F2E6908F3006A08F4008A15F2
:102C80000A120F258A150A126023FF01831203130B
:102C90006C087F028A110A16031D512E6B088316D9
:102CA00025020319582E0318582E8A150A12C22518
:102CB000831203138A110A16051A282D8A150A127F
:082CC000CB268A110A16282D0B
:02400E007A3FF7
:00000001FF
